:030000000210DB10
:03000B000200A54B
:03002B000202AB23
:03005B0002040993
:030073000203E3A2
:1000800002030406080C10182030406080040608A3
:100090000C10182030406080A0C00D0D0405060D26
:1000A0000502030302C2AFC0D0C0E020620C20688A
:1000B00002419A306602415AE47385258AC262E59C
:1000C00025F470022121206802210E758B00D0E0FA
:1000D000D0D0D290D291D292D2AF32D290D291D20D
:1000E000927406D5E0FDE53C1420E21520E10D20D8
:1000F0007D02D295307D02D29302011ED29402017C
:100100001E207D02D293307D02D29502011E758B96
:1001100000D0E0D0D0D290D291D292D2AF32758BB3
:1001200000D0E0D0D0D2AF32419AE525600A207DE0
:1001300002C290307D02C292D291419AE5256002BE
:10014000C291207D02D292307D02D290419AE52563
:10015000600A207D02C292307D02C290207D02D2D0
:1001600090307D02D292419A207D02C293307D026E
:10017000C295207D02C295307D02C2937406D5E0FF
:10018000FDE525600A207D02C290307D02C292D238
:1001900091419A207D02C293307D02C295C294742F
:1001A00006D5E0FDE525600A207D02C290307D0283
:1001B000C292D291419AC294207D02C293307D02B4
:1001C000C2957406D5E0FDE5256002C291207D024E
:1001D000D292307D02D290419AC294207D02C29583
:1001E000307D02C2937406D5E0FDE5256002C29120
:1001F000207D02D292307D02D290419A207D02C2AF
:1002000095307D02C293C2947406D5E0FDE5256069
:100210000A207D02C292307D02C290207D02D290DF
:10022000307D02D292419A207D02C295307D02C279
:1002300093207D02C293307D02C2957406D5E0FD05
:10024000E525600A207D02C292307D02C290207DA9
:1002500002D290307D02D292419A30723DE53C202C
:10026000E21A20E129207D02C293307D02C295204E
:100270007D02C295307D02C29302029A20E1E620FF
:100280007D02C293307D02C295C29402029AC2944A
:10029000207D02C295307D02C293E525F4F58A7572
:1002A0008B00D262D0E0D0D0D2AF32C2AFC2AD5359
:1002B000E6EFC0D0C0E0D2D3D2AFC2CEE52960070E
:1002C0002074461529610978007900E580307E01A7
:1002D000F430E70278FF53DACF207E0343DA203090
:1002E0007E0343DA10C2D8C271E580307E01F4305B
:1002F000E70279FFC3E89970CE30610375291820B1
:1003000074037529188859D270E52A6004152A618A
:100310001920740543DA01C2D82070026180A859FF
:10032000206102C2702074367982B70431C3E89428
:10033000F0400374F0F8E8C4540F28F87984B70348
:1003400002615EC313C3138721200802C313200A6E
:1003500006C3C898F8615E28F8500374FFF8882235
:10036000306915E5222408F52250037522FFC3E504
:1003700022955E4003855E227882B6041885222489
:10038000A824C3E524955E4002A85EC3E8956040BA
:1003900002A8608825C3E52594404002D26420CF9E
:1003A0000CD0E0D0D0C2D343E610D2AD32C2CF7869
:1003B00001E52960053074021529C3E5599401400F
:1003C00005755C0061D7755D00756400E55C24010E
:1003D000F55C5003755CFFD0E0D0D0C2D343E6108B
:1003E000D2AD32C0D0C0E0C2AF53917F53E67FC2DE
:1003F00060759100C3E49550F594E49551F59575B9
:100400009104D0E0D0D0D2AF32C2AF53E6EFC2AD4C
:10041000C0D0C0E0C0F0D2D3D2AFA8FBA9FCC2D8F4
:10042000307102817053DACF207E0343DA10307EC0
:100430000343DA20D271E580307E01F420E70281A7
:100440004788268927C1AC53DACF207E0343DA20C0
:10045000307E0343DA10C2D8C271307402C198787A
:1004600000E580307E01F430E702C1988859C17FF1
:0F04700053DACF207E0343DA20307E0343DA10C5
:10047F00C271206102A14053DACF207E0343DA100C
:10048F00307E0343DA20C2D8D27188548955C3E82D
:10049F009552F8E99553F9E4FB7E027A00C3E8948C
:1004AF008CE994005005755800A130C3E894C8E951
:1004BF0094005008E4D2E4FB7A0AA10DC3E89468D3
:1004CF00E994015008E4D2E3FB7A0FA10DC3E8943D
:1004DF00D0E994025008E4D2E2FB7A1EA10DC3E8E2
:1004EF0094A0E994055008E4D2E1FB7A3CA10DC336
:1004FF00E89498E994085008E4D2E0FB7A787E00FB
:10050F00C3E89556FCE99557FD30E708ECF4240154
:10051F00FCEDF4FD755800C3EC9AED9E5003755831
:10052F000188568957A854A955885289537802C112
:10053F007FC3E89526F8E99527F9307C02C163302F
:10054F007B02C163307A02C15C207502A163E9FDB1
:10055F00E8FCA182E9C313F9E813F8307902C15C12
:10056F00E9C313F9E813F8307802C15CE9C313FD4E
:10057F00E813FC206126C3EC941CED94024002A109
:10058F0099ED7018C3EC94C850120528C3E5289450
:10059F000A5002C198755900D270C198E5286002BF
:1005AF0015287400207F0B7888E67896B4030278BC
:1005BF009EE624FAFEE43400FFC3EC9EFCED9FFDA3
:1005CF0092087888E6B40327A2085009207D20C23C
:1005DF00AFD27DA1EB307D17C2AFC27DD290D29149
:1005EF00D292C293C294C295206902D26BD2AFA2AB
:1005FF00085017E6B4030DECF42401FCEDF43400BD
:10060F00FD02061978007900C1637888E6B40315F6
:10061F00EC33FCED33FDC3EC940AFCED9400FD507C
:10062F00047C007D00C3EC94FFED9400400678FF3E
:10063F007900C163EC856FF0A4C5F0A2F733F879A8
:10064F0000400302067F78FF790002067FE9C3139B
:10065F00F9E813F8307C0EE9600278FFC3E813382D
:10066F00F8E43400F9C3E894FFE99400400278FFFE
:10067F008859D270206102C198741FF4552F4BF521
:10068F002FC274E42B7002D274752918307403755D
:10069F00290A306102C1AC20740353DAFE752A06B1
:1006AF00307403752A0AD0F0D0E0D0D0C2D3D2ADC7
:1006BF0043E6103279010206E179030206E1790A75
:1006CF000206E1791E0206E179640206E179C802A9
:1006DF0006E17817E4D5E0FDD8FAD9F6227A147B33
:1006EF00780207087A107B8C0207087A0D7BB40218
:1006FF0007087A0B7BC8020708AC2575250179021C
:10070F00B27DE4C294D5E0FDE5256002C291D5E04B
:10071F00FDD291D5E0FDD294D5E0FDE525600A200C
:10072F007D02C290307D02C292E570D5E0FD207D42
:10073F0002D290307D02D2927496D5E0FDD9C1EAF3
:10074F00F8D5E0FDD8FBDBB1C2948C2522C37C0029
:10075F007D0075F00005F0EA33FAEB33FB50F6EB52
:10076F0013FBEA13FAC3E9FFE8FEE89AF8E99BF9ED
:10077F005004EFF9EEF8B3EC33FCED33FDD5F0DFB9
:10078F00EDF9ECF822E889F08A20D2D4F8A9F07BB1
:10079F000030F70B7BFFF42401F8E9F43400F9E89B
:1007AF008520F0A4ADF0F8E98520F0A4AFF0FEEDC0
:1007BF002EF974003FFA7C04C3EA13FAE913F9E83F
:1007CF0013F8DCF48BF030F70AE8F42401F8E9F4BD
:1007DF003400F9E889F0C2D4F8A9F0227882B6047F
:1007EF0003020848C3E5599401400302081085220B
:1007FF0024E4F53EF53FF540F541F542F547020893
:10080F00487882E6FC754701E522F523783879C7E9
:10081F00AA3AAB3BC3EB13FBEA13FAEC146013C316
:10082F00EB13FBEA13FAEC14146007C3EB13FBEAA8
:10083F0013FA12075C883E893F22E5476034C3E50F
:10084F003E9523F8E53F9400F9500CC3E89480E9F6
:10085F0094FF401602087DC3E8947FE9940050038B
:0E086F0002087D787F790002087D788079FF8D
:10087D008843894422E5476058E5432540F8E5441F
:10088D003541F9854420E4300701F43542FA30E76B
:10089D0009C3EA94F040150208BFC3EA940F500350
:1008AD000208BF78FF79FF7A0F0208BF7800790040
:1008BD007AF0C3E524955E5006E524600901D8E57C
:1008CD004420E70D01D8E54430E706884089418A88
:1008DD004222E547700302094378A1E6FAC3E543D6
:1008ED0033F8E54433F9120794E930E70BC3E89484
:1008FD0080E994FF4013211AC3E8947FE9940050D6
:10090D0002211A787F7900211A788079FFE820E793
:10091D0015C3E52398F84009C3E894014003020983
:10092D00417801020941E8F424012523F84003022E
:10093D00094178FF884522E54770030209A678A290
:10094D00E6FAA841A942120794E930E70CC3E894EE
:10095D0001E994FF401602097DC3E894FFE9940074
:10096D00500302097D78FF790002097D780179FF36
:10097D00E920E715C3E54598F84009C3E89401401F
:10098D00030209A478000209A4E8F424012545F81E
:10099D0040030209A478FF88242278FFC264E52D64
:1009AD005406702FD264C3E53B940A4009C3E52574
:1009BD0094405002C264E53B601974FF853BF0849E
:1009CD008537F0A4F8C5F0600278FFC3E895615053
:1009DD0002A8618860227883E6F520120F0175E880
:1009ED00901206C375E890E5E820ECFBA8BDA9BE02
:1009FD00120F97756B30756C00C3740013FD743056
:100A0D0013FC74302CFC74003DFDECFAEDFBC3E8D7
:100A1D009AE99B4014E56B2430F56BE56C3400F5D9
:100A2D006CEA2CFAEB3DFB80E5AE6BAF6CC3E56C6D
:100A3D0013F9E56B13F8C3E913F9E813F8E56B281F
:100A4D00F569E56C39F56A7A03C3E913F9E813F82A
:100A5D00DAF7AA201A7009756B00756C00020A7D11
:100A6D001AEA6008EE28FEEF39FFDAF88E6B8F6C0C
:100A7D002275E890227883E6FFE5E820ECF7A8BD23
:100A8D00A9BE056DC3E56D94084052756D00E9FA78
:100A9D0079A0E76044EA7007E56E601B020AB8C3EF
:100AAD00E8956E6010E56E5006600C14020AC404E1
:100ABD0060F9020AC4E56EF56EC3946D401B755E58
:100ACD00C0C394044013755E80C39404400B755EDF
:100ADD0040C394044003755E0075BB0622EFC394BA
:100AED0001601BC3E894FFE994035012C3E8956BB2
:100AFD00E9956C5009E55E601A155E020B20E55E06
:100B0D00F46010055E7888E6B40308E55E240440C1
:100B1D0002F55EA85EC3E524985002A824C3E895AB
:100B2D005F400AA85FE55FF46003855F5E7982B779
:100B3D000402614BC3E895604002A8608825E56D0D
:100B4D00B4070375BB1022743279A387F0A4C5F0E6
:100B5D00A2F733F8C3E8955E4002A85E8822882488
:100B6D008825886122753A00753B7F2275C820A8BB
:100B7D00CCA9CD75C824AA38AB3988388939C3E8D2
:100B8D009AF8E99BF9AA3AAB3BAC3AAD3B7E047FB0
:100B9D0002C3EB940440021E1FC3EB940840021ED7
:100BAD001FC3ED13FDEC13FCDEF7C3EA9CFAEB9DBE
:100BBD00FBEF6009C3E913F9E813F8DFF7EA28FA48
:100BCD00EB39FB8A3A8B3B400122753AFF753BFFAF
:100BDD002230600261DE854C50854D51D26043E676
:100BED0080227892E6FFC3E535948240010FC3E57C
:100BFD003594A040010FC3EF940640027F057E029D
:100C0D001E3072010EC3E53B940350060E0E30727A
:100C1D00010EC3E53B940250060E0E3072010EA973
:100C2D003BA83A7A04C3E913F9E813F8DAF7C3E8F5
:100C3D009EF8E99400F94009C3E89402E994005044
:100C4D00047802E4F9E9FBE8FAC3E913FDE813FCC3
:100C5D00884C894DC3EF94036037EF20E00DE82CED
:0F0C6D00F8E93DF9ECFAEDFB020C8BE828F8E909
:100C7C0039F9C3E89402F8E99400F97A02E4FBC369
:100C8C00EF9403400D8A4E8B4F884889498C4A8DCE
:100C9C004B22884E894F8A488B498C4A8D4B223087
:100CAC00600281ABD26043E680E52D54066027A834
:100CBC003AA93BE53494085006E820E002A94D75AA
:100CCC009100C3E498F594E499F595759104D2607C
:100CDC0053917F43E68022D265753D00752000025A
:100CEC000CF6D265753D00752040E52D540660026A
:100CFC00C265D2AF206005E53D60012278017A0221
:100D0C00C3E53B940540027802C3E53B940A4002DC
:100D1C007803C3E53B940F40027A03306904781ED4
:100D2C007A01206007E53D6003D2AF22D2AF00000C
:100D3C00C2AFC3E53BFB940F40027B0FEB04307357
:100D4C00012320620123F93069027982E58BC39972
:100D5C0040D0053DEAFBE59BF45440B52004DBF69E
:100D6C00A19220650281F6C265759100AE3AAF3B47
:100D7C00C3E49EF594E49FF595759104D26053916C
:100D8C007F43E68081F630650281F6D895D2AF229A
:100D9C0030690B0534206016753400020DBA2060E2
:100DAC000D20650A206B071581158102159722A865
:100DBC004EA94F75910053917FC3E498F594E49933
:100DCC00F595759104854850854951D26043E6806C
:100DDC002278003064053065027801E53575F0073E
:100DEC00A4F9E5F028F5F0E9A2F013A2F113A2F2B0
:100DFC0013F535C394785003753578C3E5359536BE
:100E0C004008D266D290D291D292306002C116853F
:100E1C004A50854B51D26043E68022C2AFC293C286
:100E2C0094C29530720B9001FC7406D5E0FD020E55
:100E3C003D207D02D293307D02D295759F11753C79
:100E4C0002020F7CC2AF207D02D292307D02D29082
:100E5C003072179001D9C294207D02C295307D0268
:100E6C00C2937406D5E0FD020E7990013C30620607
:100E7C00E5256002C291207D03759F21307D0375AD
:100E8C009F01753C03020F7CC2AFC293C294C29502
:100E9C0030720B9001B67406D5E0FD020EAA207DCF
:100EAC0002D295307D02D293207D03759F01307D57
:100EBC0003759F21753C04020F7CC2AFD291307236
:100ECC0017900193207D02C293307D02C295C2948B
:100EDC007406D5E0FD020EE790012A30620EE5257E
:100EEC00600A207D02C290307D02C292759F1175FE
:100EFC003C05020F7CC2AFC293C294C29530720BF8
:100F0C009001687406D5E0FD020F17D294207D0382
:100F1C00759F21307D03759F01753C06020F7CC2C5
:100F2C00AF207D02D290307D02D29230721F90029F
:100F3C0027207D02C293307D02C295207D02C2958E
:100F4C00307D02C2937406D5E0FD020F5C90014E19
:100F5C0030620EE525600A207D02C292307D02C20D
:100F6C0090207D03759F01307D03759F21753C0199
:100F7C00306B13120F977406D5E0FD7406D5E0FDA7
:100F8C00D293D294D295C266D2AF22900128D2903D
:100F9C00D291D292C293C294C295C26222788076C8
:100FAC00090876090876040876010876030876FFA6
:100FBC00087608087601087601087601788C7601A7
:100FCC000876FF0876FF0876FF0876FF0876FF089C
:100FDC0076030876FF0876FF0876FF0876250876F4
:100FEC00D00876280876500876040876FF08760232
:100FFC0008760008767A0876FF087601227887E66C
:10100C00FFC2727888E6C394036008C27DE630E1C3
:10101C0002D27DC27E7889E630E102D27EC3EF94A3
:10102C00026008758E01D27302103C758E00C2737B
:10103C00227880E6149000809378A1F67881E614EB
:10104C009000809378A2F6120F97227886E614907F
:10105C00008D9378A3F6120F972222789CE67536B2
:0D106C00FF75370CB402067536A075370A03
:10107900B4030675368275370522227896E6FA7822
:1010890097E6FB307F047A007BFFC3EB9AFCC3949D
:101099008250027C82756F00056FEC856FF0A4C3E6
:1010A900E5F0948040F222D27F11841206D27A00B0
:1010B9007B007C101206C8E5592AFA74003BFBDC58
:1010C900F37C04C3EB13FBEA13FADCF7FEC27F11CE
:1010D9008422E5EF20E6037520000520903FFFE517
:1010E90020146006901DFF1460009304600375EFDF
:1010F90012C2D353D9BF7581C043FF801206C3758D
:10110900EF0243B203E5B3240420E702F5B3120F5B
:10111900977580FF75A40075F19175D47F75900757
:1011290075A53F75F2FF75D50075A60175E24112E7
:101139000FA91215C878988670C2AF1206DC12067C
:10114900EC1206D21206F31206D21206FA1206D2CF
:10115900C2AFE4F8F6D8FD78C879C8308707D9FB5B
:10116900D8F7021C00120FA91215C81109113D1157
:1011790057116611671183118478988670120F9739
:1011890075885075891275C82475910475D840758C
:10119900A82275B80275E690759B80759D0075D17A
:1011A9000E75BC5875BB0675BA1175E8801206C371
:1011B900D2AF1209E343DA01C2D8C2711206DC7553
:1011C9003001D2617B037A0CE55870067A0CDB0298
:1011D90021591206D22070022159C270E559C394CF
:1011E9000240E3E52F541F855B5AF55BB55AD7DA00
:1011F900D7C26153DACF207E0343DA20307E03431E
:10120900DA10C2D8C271C2757528001206D73074B7
:1012190009C3E528940A4002D2751206C87802303B
:1012290074027800C3E5599840F0C2AF1206EC1277
:1012390006EC1206ECD2AF1206DC7546007888E699
:10124900B4030261221206C8788CE6C394015003E4
:10125900021322E530C3940150030213222074358E
:10126900C3E55994FF5003021322C2AF120701D2FA
:10127900AF1206D7C3E559940150EFC2AF1206EC7D
:101289001206CD1206ECD2AF1206D7C3E55994FF68
:1012990040E90217707F02D27F11841206D7C2AFCC
:1012A900C27F1184AE59C3E559947FD2AF407412FD
:1012B90006C3C2AF120701D2AFDFDC11B0C3EE948F
:1012C900057897F61206DC12160A1216F37F0AD26F
:1012D9007F11841206D7C2AFC27F1184AE59C3E50C
:1012E90059947FD2AF50E61206C3C2AF1206EC1270
:1012F90006CD1206ECD2AFDFD611B0EE24057896F2
:10130900F61206DC12160A1217221206D71184C326
:10131900E55994FF40F4021770C3E5599546400317
:101329008559461206D778017988E7B4030278050A
:10133900C3E5599840024146C2AF1207011207019D
:10134900120701D2AF1206DC753000E4F531F5322F
:101359000531E531F470390532789AE67819146067
:1013690012783214600D787D14600878FA146003DD
:10137900753200C3E53298401715327531B4789942
:101389008670C2AF120701D2AF789886701206D75D
:101399001206CDE5297005307402215978012074AF
:1013A900027806C3E5599840A77888E6C394036094
:1013B900031206D7E52970022159C2AF120F97E42B
:1013C900F522F523F524F525D2AF78858662F53E19
:1013D900F53FF540F541F542F56DF547F52CF52D4D
:1013E900F535120B72756D0875BB101206C3120A1A
:1013F9007EE5E820ECFBA8BDA9BEE97001F8886E7E
:10140900120A82756D0875BB107887E6FE7602119F
:10141900097887EEF6C2AF755EFF120B5485225E1E
:1014290085225F852260D2AF752201752401752559
:1014390001855D64756501D268D269753400120F42
:1014490001120F2B120B72120B79120BEF0214649B
:10145900120F971109756D0075BB06120CEE120D6E
:0D1469009C120DBB1207EB120DDD120E27B9
:10147600120B79120BDE120BEF120CAB120CE312ED
:101486000D9C120DBB1208491209A7120DDD120E92
:1014960050120B79120BDE120BEF120CAB120CEE84
:1014A600120D9C120DBB120882120DDD120E941243
:1014B6000B79120BDE120BEF120CAB120CE3120DB2
:1014C6009C120DBB1208DF120DDD120EC6120B792F
:1014D600120BDE120BEF120CAB120CEE120D9C125D
:1014E6000DBB120944120DDD120F01120B79120BFE
:1014F600DE120BEF120CAB120CE3120A7E120D9CDD
:10150600120DBB120A82120DDD120F2B120B79126D
:101516000BDE120BEF120CAB306938206B35856190
:101526005E85615F855D6475650179327A0AC3E51A
:1015360034994012C269D26A8A3385615E755FFF4B
:10154600756020021559C3E55994014003021464DD
:10155600021597306A1E206B1BE533147007C26AAA
:10156600755EFF8159F533C3E559940140030214B2
:1015760064021597C3E55C94FA5016307404E529A5
:10158600600FC3E53B78F0306B02786098500281BB
:1015960064C2AF120F977887E6FE76021109788744
:1015A600EEF6E4F522F523F524F525F562C268D2B8
:1015B600AF1206C3120F97307406E529700221593F
:1015C6006154901A0D782012164CE520B4550CA3E0
:1015D60012164CE520B4AA030215EA120FA9121638
:1015E6000A021609901A0378807B0A12164CA30881
:1015F600DBF9901A0F788C7B1512164CA308DBF9D1
:10160600901A2422C2AF12168B121665901A007415
:101616000D121651A37402121651A3741312165109
:10162600901A0378807B0A121650A308DBF9901AE9
:101636000F788C7B15121650A308DBF912169E1232
:10164600167C901A2422E493F622E6438F01538FE8
:10165600FD75EF0275B7A575B7F1F0538FFE2243FE
:101666008F02438F0175EF0275B7A575B7F1901A12
:101676000DF0538FFC22901A0D7455D151901A0E0D
:1016860074AAD151227A3079D07820901A40D14C60
:10169600E520F709A3DAF7227A3079D0901A40E7E5
:1016A600D15109A3DAF922AB71A872BB0102798084
:1016B600BB02027981BB03027982BB04027984BB37
:1016C60005027983BB06027986BB07027992BB08BD
:1016D600027987BB0902799CBB0A027988BB0B0297
:1016E6007989E8F7227C051206DCDCFB22C2AF1200
:1016F60006EC1206F31206FA1207011206CD1206BE
:10170600EC1206F31206FA1207011206CD1206ECC7
:101716001206F31206FA120701D2AF22C2AF12075F
:10172600011206FA1206F31206EC1206CD12070192
:101736001206FA1206F31206EC1206CD1207011271
:1017460006FA1206F31206ECD2AF22AE71AF72C2DF
:10175600AF1206EC1206EC1206EC1206CDDEF21201
:1017660007011206CDDFF8D2AF22D1F3D1EBD1EBD0
:10177600757101757201757300F1517C05AD5912D1
:1017860006DCC3ED955970F5C3E5599401400AC3CB
:10179600E55994FF40320217ACD1ADD10AD1F3C25C
:1017A600AF75EF12D1EBDCD50573C3E57394035027
:1017B6000280C6D1EB0572E5711490009A93F80881
:1017C600C3E57298500280AED1EBD1EB0571C3E54B
:1017D60071940C5002809C120FA9D10AC2AF75EF0A
:0317E60012D1EB32
:101A00000D02130909040103FF0801010155AA0190
:101A1000FFFFFFFFFF03FFFFFF25D0285004FF0259
:051A2000007AFF01FF48
:101A400023506F6C61726973546472383041232083
:101A500023424C48454C4923463333302320202031
:101A60002020202020202020202020202020202076
:101C0000C2AFC2D353D9BF7581C043B20343FF8073
:101C1000752438752503B1BF75EF0275E24043F1B5
:101C20008053A47FD287780379E67C1075220075F3
:101C30002300901DCC7B0675249875250130870202
:101C4000813D208708D8FBD9F9DCF781AD308708C2
:101C5000D8FBD9F9DCF781ADB17FE493A3C39A60D7
:101C6000028126DBDDB171600281267B08E493FAF4
:101C7000A3B152DBF87A30B152752200752300B15E
:101C800071EAFCEBFDC3ED94FE400EB1718A278B27
:101C900028ED30E0048A828B83B1717AC270D8C398
:101CA000ED94FE601050CEBD0022EC600675200061
:101CB0000200008100A827A9280809D804D90281B8
:101CC000C9B175EA89AAF281BB0D8199C3ED94036C
:101CD0005049EDA2E092007AC5C3E5829400E58305
:101CE000941C5093200010438F02438F0175B7A5B9
:101CF00075B7F1F030001FA827A9280809438F0104
:101D0000538FFDD804D902A11689AAE275B7A5752B
:101D1000B7F1F0A3A103538FFC81757AC1BD030C09
:101D2000E493A3FAB136DCF8B12E81758177AA224B
:101D3000AB23B152EBFAEA6222752608C3E52313FE
:101D4000F523E52213F52250066323A0632201D573
:101D500026EAB1BFB1BF75260AEAF4200102D28794
:101D6000300102C287B1BFC3134002C201D526EBC6
:101D700022B175EAFB208702A175308702A17A752E
:101D80002608AE24AF25C3EF13FFEE13FEB1C3B197
:101D9000BFC3EA133087024480FA30E703632201AD
:101DA000C3E52313F523E52213F52250066323A090
:101DB000632201D526D9E52265236523F52222AECB
:101DC00024AF250E0FDEFEDFFCD20122424C486517
:0A1DD0006C6934373132F33006013C
:00000001FF
